:020000040000FA
:100000006400831600308600831286019A0108304E
:1000100097008601990195011830940064006020D2
:1000200010080839031D3628970B1E286400083075
:1000300097001A08013E07399A0099016400FF30C1
:100040008600602010080139031D0E281508031DC5
:100050002E285420940B0E28FF30950064000030A9
:1000600086004820FF30860048200E28640060206B
:1000700010080239031D09286020100804390319EB
:100080004628602010081039031D092871200E2809
:1000900064006F309200FF30930064000000930B07
:1000A0004D28920B4B28080064001F309200FF304F
:1000B000930064000000930B5928920B5728080006
:1000C000640005081F3990003F3092006400920BD5
:1000D000662805081F39100203190800FF30900038
:1000E00008006400862098001908031D7B28180862
:1000F0009600990A712818088600482019081602E7
:10010000031D842899010800990A080064001A0850
:10011000031D9B28190882070E340134023404346D
:1001200008341034203440348034403420341034C7
:100130000834043402341A08013C031DB22819089B
:100140008207103400340134033407340F341F3471
:100150003F347F34FF347F343F341F340F3407344F
:10016000033401341A08023C031DD72819088207FA
:100170001E3400340134033407340F341F343F3449
:100180007F34FF34FE34FC34F834F034E034C034CF
:100190008034C034E034F034F834FC34FE34FF34BE
:1001A0007F343F341F340F340734033401341A08CA
:1001B000033C031DF4281908820716340034013467
:1001C000023405340A34143428345034A034403412
:1001D0008034003480344034A03450342834143413
:1001E0000A340534023401341A08043C031D092979
:1001F000190882070E340134803402344034043448
:1002000020340834103408342034043440340234A8
:1002100080341A08053C031D202919088207103470
:100220000934063412340C3424341834483430344D
:10023000903460344834183424340C341234063486
:100240001A08063C031D3329190882070C340034B0
:10025000FF340034E7340034C334003481340034D4
:10026000C3340034E734190882070C3400340334F3
:1002700000340C34003430340034C03400343034B2
:0402800000340C3406
:02400E00FF3F72
:00000001FF
